:0600000000308A00052813
:1000080009000A128A1151298030831603139F00B0
:10001800453083129F00000000009F149F1812288B
:100028001E08A30083161E088312A2002308FF00DF
:100038002208FE0008008030831603139F00413019
:1000480083129F00000000009F149F1829281E0893
:10005800A30083161E088312A2002308FF002208AB
:10006800FE0008008301AC002C1C3C2807163D2824
:100078000712AC1C41288716422887122C1D4628D7
:10008800071747280713AC1D4B2887170800871345
:10009800080034308301A4000230A500B308031D12
:1000A80058288D30A400A501330B5D28BC30A4006E
:1000B800A5013308023A031D6428EB30A400A5010A
:1000C8003308033A031D6C281A30A4000130A50038
:1000D8003308043A031D74284930A4000130A500F0
:1000E8003308053A031D7C287830A4000130A500A8
:1000F8003308063A031D8428A730A4000130A50060
:100108003308073A031D8C28D630A4000130A50017
:100118003308083A031D94280530A4000230A500CE
:100128003308093A031D9C283430A4000230A50086
:1001380033080A3A031DA4286330A4000230A5003E
:1001480033080B3A031DAC289230A4000230A500F6
:1001580033080C3A031DB428C130A4000230A500AE
:1001680033080D3A031DBC281330A4000330A50042
:1001780033080E3A031DC4283C30A4000330A50000
:1001880033080F3A031D08006530A4000330A500AA
:10019800080031308301AD008B13AE012E082D0706
:1001A800840083130008AF002E080A128A11232244
:1001B8000A128A11AE0A03302E02031CD2288B17AA
:1001C800080083010808AC00AC1FEC28A001A00AB5
:1001D800A008031DAC1B0800A0010808AC0070397A
:1001E800703A031DFB282C080F39A10008002C08C1
:1001F8007039603A031D082921083106031D0800DB
:100208002C080F39B200CD282C087039503A031D3C
:10021800080021083106031D08002C080F39B30017
:100228004D20CD2831308301AC008B13AD012D0852
:100238000A128A1143220A128A11FE002D082C077D
:10024800840083137E088000AD0A03302D02031C4E
:100258001B298B17080083010610861087100712C8
:10026800871207138713113083168500FC30860028
:100278000D308700FF308800890080309F000330F0
:100288000317880089014130831203139F008B17DD
:100298000B17A001A00AA10108002F2116214D204B
:1002A8006400071D871D5D29320836208610061454
:1002B800032A871D071D6529320836200610861473
:1002C800032A061086100F303620E5200A128A11FC
:1002D8001F207E08AA007F08AB002508FF0024081D
:1002E800FE00F630FE070318FF0AFF30FF072B0851
:1002F8007F02031D81292A087E02250803189B29ED
:100308002B02031D892924082A0203189A29A70108
:1003180087140000871000000000000000000000A3
:10032800A70A0A3027020318032A8C2925082B025A
:10033800031DA02924082A020318032A00302B02CF
:10034800803003192A020318B829A701871400006E
:10035800871000000000000000000000A70A3230EB
:1003680027020318032AAA2901302B020030031997
:100378002A020318CC29A70187140000871000005F
:1003880000000000A70A643027020318032AC029C6
:1003980002302B02003003192A020318E029A701B2
:1003A800871400000000871000000000A70AC8306A
:1003B80027020318032AD42902302B02803003199C
:1003C8002A02A7010318F62987140000000000007C
:1003D8000000871000000000A70AC8302702031891
:1003E800032AE82987140000000000000000871095
:1003F80000000000A70AC8302702031CF6290820BD
:100408007E08A8007F08A90000302902EC300319F3
:100418002802031C542906108610A7016400A601AF
:100428000000000000000000A60A64302602031C39
:10043800142AA70A6430270203185429122A8301B0
:10044800B000831603178C18252A8312031330086B
:1004580003178D0003132F0803178C0083168C13C2
:1004680003108B1B03148B130C1555308D00AA3009
:100478008D008C140C1103188B178301080083015D
:10048800AE00831603178C18452A831203132E080F
:1004980003178D0083168C130C1483120C08031396
:1004A800080083012708260403190800A608031971
:0E04B800A703A60327082604031908005A2AE2
:02400E00FC1F95
:10420000020008000900000000000000000000009B
:10421000000000000000000000000000000000009E
:10422000000000000000000000000000000000008E
:10423000000000000000000000000000000000007E
:10424000000000000000000000000000000000006E
:10425000000000000000000000000000000000005E
:10426000000000000000000000000000000000004E
:10427000000000000000000000000000000000003E
:10428000000000000000000000000000000000002E
:10429000000000000000000000000000000000001E
:1042A000000000000000000000000000000000000E
:1042B00000000000000000000000000000000000FE
:00000001FF
